:020000040000FA
:1000000083018B018A012728F0000308F1000A0808
:10001000F2000408F3008312031383138A01B9303A
:1000200081000B112408081D18280530A1001A288A
:100030000130A100002586002108A0077308840074
:1000400072088A0071088300F00E700E0900031315
:10005000831283138525E025B9308100A0308B0001
:100060005E204D218C1E312830280C1E3528990029
:100070008316981C3928831208008C1E3D28981C72
:100080004428181218163D28181D48281A083D281B
:100090001A080800AB002B0E0F39542035202B080E
:1000A0000F3954203520080003138312AD000A30A5
:1000B0002D020318073E0A3E303E0800533035201B
:1000C000653035206C303520653035206330352083
:1000D00074303520203035204E3035206F303520BB
:1000E0002E30352028303520313035202C30352049
:1000F000323035202C303520333035202C3035202F
:10010000343035202C303520353035202C3035201A
:10011000363035202C303520373035202930352009
:100120000D3035200A3035200230BE003D20D5008C
:10013000550835205508313A031DA028CC20B72892
:100140005508323A031DA628DA20B7285508333A55
:10015000031DAC28E820B7285508343A031DB228FF
:10016000F620B7285508353A031DB72804210800A2
:10017000C501C601D301D401CA010A30CC003D300B
:1001800084000008CA001221840ACC0BC12853083D
:10019000C5005408C60008004A30BF004730C00000
:1001A0003630C1005930C2004930C3004730C40066
:1001B000B82008004830BF004530C0004C30C100B6
:1001C0004C30C2004F30C3002130C400B8200800BA
:1001D0005330BF004830C0004930C1004E30C2002B
:1001E0004530C3004E30C400B82008004A30BF007C
:1001F0004130C0005030C1004130C2004E30C30019
:100200002130C400B82008004130BF004230C00097
:100210004330C1004430C2004530C3004630C40002
:10022000B82008000830C9000310CA0DD40DD30D42
:10023000031C1E291030D3062130D406C90B142903
:100240000800CD01CE0152100A30D0003D308400AC
:100250000008CF003E21840AD00B28294D084A20EF
:100260004E084A20CD08031D3A29CE08031D3A291D
:1002700052103D29CD01CE01521408000830D100A2
:100280000310CF0DCE0DCD0D031C4A291030CD0625
:100290002130CE06D10B402908003A30B0000D3095
:1002A000AF003008840000086521B00AAF0B512967
:1002B00008003E30C8000730C700480884003D20D1
:1002C0008000C80AC70B5D290800B2000830B500DD
:1002D0000810881008148814B21F7029031071299F
:1002E0000314B70DB60DDA2588100130B706371C98
:1002F000081137180815DA2508108814B20DB70D43
:10030000B60DDA2588100130B706371C08113718EA
:0A0310000815DA25B50B6A2908006C
:100A000005308A0020087F398207803486348C3490
:100A1000933499349F34A534AB34B134B634BC34F8
:100A2000C134C734CC34D134D534DA34DE34E23492
:100A3000E634EA34ED34F034F334F534F834FA348F
:100A4000FB34FD34FE34FE34FF34FF34FF34FE3417
:100A5000FE34FD34FB34FA34F834F534F334F03436
:100A6000ED34EA34E634E234DE34DA34D534D134E9
:100A7000CC34C734C134BC34B634B134AB34A5340F
:100A80009F34993493348C34863480347A3474347B
:100A90006D34673461345B3455344F344A344434F4
:100AA0003F34393434342F342B34263422341E343A
:100AB0001A341634133410340D340B34083406341D
:100AC0000534033402340234013401340134023475
:100AD000023403340534063408340B340D34103436
:100AE000133416341A341E34223426342B342F3463
:100AF000343439343F3444344A344F3455345B341D
:100B0000613467346D3474347A340313831283167A
:100B1000003085000030860080308700003088007B
:100B2000003089008312003085008030860000305C
:100B300087008030880000308900831681120112FE
:100B40008115831283168130990024309800831216
:100B500090309800FF30920083166130920083122B
:100B60002310A001A2010130A100A3010130A400C3
:100B70008330A6000530A500AB01AD01D201FA30EB
:100B8000BA00F330BB002030BC000630BD0000309E
:100B9000BE00BF00C000C100C200C300C400080006
:100BA0008C108C1CD12D08000430A700D025A70B79
:100BB000D62D08000530A800D025A80BDC2D080094
:100BC0001430A900D025A90BE22D08003A30B0005E
:100BD0000D30AF003008840000084A20B00AAF0B87
:040BE000EA2D0800F2
:02400E00723FFF
:00000001FF
